:100000007FC0000099C0000097C0000095C00000AC
:1000100093C0000091C000008FC000008DC00000A0
:100020008BC0000089C0000087C0000053C60000DC
:1000300083C0000081C000007FC000007DC00000C0
:100040007BC0000079C0000078C0000075C00000CF
:1000500073C0000071C000006FC000006DC00000E0
:100060006BC0000069C0000067C0000065C00000F0
:1000700063C000001201100102000008EB034420DD
:1000800001000102DC0109023E00020100C0320948
:1000900004000001020201000524001001042402F2
:1000A000060524060001070582030800FF09040174
:1000B00000020A0000000705040210000107058382
:1000C00002100001040309041803440065006100E4
:1000D0006E002000430061006D0065007200610049
:1000E00000001C034C005500460041002000430066
:1000F000440043002000440065006D006F000000D4
:1001000011241FBECFEFD2E0DEBFCDBF12E0A0E0D2
:10011000B1E0E8E6FCE102C005900D92A833B1071A
:10012000D9F712E0A8E3B2E001C01D92A937B107E8
:10013000E1F7C3D00C94320E63CF1F920F920FB62B
:100140000F9211248F939F9388E59EE990938500E9
:1001500080938400809138029091390201969093A7
:100160003902809338029F918F910F900FBE0F90AC
:100170001F901895E1E8F0E080818360808388E536
:100180009EE99093850080938400EFE6F0E0808103
:100190008160808308958BB180668F7B8BB90895D1
:1001A0008BB180668F7D8BB9089580E292E00C94CC
:1001B000570A80E292E00E94070A80FD02C090E2A6
:1001C00001C090E48BB19095806698239BB9089507
:1001D00084B7877F84BF88E10FB6F894809360006E
:1001E000109260000FBE80E090E020E80FB6F89417
:1001F00020936100809361000FBE8AB180668AB946
:100200008BB180668BB957D557985F9AB3CF0F9350
:100210001F9380913A0290913B026AE070E00E9445
:10022000100B062F80E090E00E944B0D20913C02C5
:1002300030913D0224503040132F81E090E0632F35
:100240000E944B0D60913C026450060F82E090E0EA
:100250000E944B0D100F83E090E0612F0E944B0D28
:100260001F910F910895D3CF08951F93DF93CF93DC
:1002700000D0CDB7DEB710914C0280E060E070E0B6
:10028000C4D28CE49DE120E931E0F9013197F1F726
:100290000197D9F7812FBE016F5F7F4FF5D2882379
:1002A00019F020E938EE02C029813A81C9010F9086
:1002B0000F90CF91DF911F9108952F923F924F920F
:1002C0005F926F927F928F929F92AF92BF92CF92E6
:1002D000DF92EF92FF920F931F93DF93CF93CDB7EF
:1002E000DEB729970FB6F894DEBF0FBECDBF70DF23
:1002F00080E090E00E94430DD82E90E06AE070E02C
:100300000E94FE0A90933B0280933A0281E090E0C3
:100310000E94430DF82E182F00E010933D02009329
:100320003C0282E090E00E94430DE82E90E0082B12
:10033000192B0C5F1F4F10933D0200933C02FD0CE4
:1003400083E090E00E94430DFE0C8F1561F086E97A
:1003500090E090933B0280933A0284E090E0909387
:100360003D0280933C0280E292E06EE372E0C0D7EF
:100370008BB180668F7D8BB97894DED28FEF8983C5
:1003800000E010E062E0E62EF12CEC0EFD1E5E01B6
:100390000894A11CB11C5AE0C52ED12CCC0EDD1E38
:1003A0002FC0C501B701A4D289818F3F11F08E3FC4
:1003B000B9F488249924AA24BB24EE24FF244EE314
:1003C000C42E42E0D42E32E0232E32E0332E2EED26
:1003D000622E21E0722E97EC492E91E0592E17C023
:1003E000D701F80183E0EE0FFF1F8A95E1F7E45B88
:1003F000FD4F8D918193AC15BD05D9F70F5F1F4F50
:1004000089818823B1F20430110559F6D2CF80E2F8
:1004100092E041D7181619060CF007C18A309105F1
:1004200019F08F33910539F580E091E06EE372E0C9
:100430000E94480B88E191E06EE372E00E94480B55
:1004400080E391E06EE372E00E94480B8AE491E061
:100450006EE372E00E94480B82E691E06EE372E088
:100460000E94480B8EE791E06EE372E00E94480B19
:100470008CE991E0D6C084379105B9F4F6DE28EE18
:100480008039920719F48AEB91E0CBC000D000D0FC
:1004900000D0EDB7FEB73196ADB7BEB71296DC927D
:1004A000CE9211975382428215C08336910501F591
:1004B00000D000D000D0EDB7FEB73196ADB7BEB7D3
:1004C0001296DC92CE9211977382628280913802EA
:1004D00090913902958384830E94370B2DB73EB7E4
:1004E0002A5F3F4F0FB6F8943EBF0FBE2DBF9DC091
:1004F0008836910561F58DB79EB708970FB6F894C9
:100500009EBF0FBE8DBFEDB7FEB73196ADB7BEB77C
:100510001296DC92CE9211972CEE31E03383228337
:1005200080913A0290913B026AE070E00E94100BC9
:100530007583648380913C0290913D020497978378
:1005400086830E94370B8DB79EB7089662C08436AB
:10055000910581F504E010E023C0C8010E94430D1D
:1005600000D000D000D0EDB7FEB73196ADB7BEB722
:100570001296DC92CE92119733822282992787FDC0
:100580009095958384830E94370B0F5F1F4F2DB783
:100590003EB72A5F3F4F0FB6F8943EBF0FBE2DBF48
:1005A00080913C0290913D0208171907B0F286E055
:1005B00092E037C0C1978930910588F5AAE0B0E094
:1005C00002C0AA0FBB1F8A95E2F7B0933B02A0932B
:1005D0003A021DDE00D000D000D0EDB7FEB7319654
:1005E000ADB7BEB71296DC92CE9211972FE032E0F3
:1005F0003383228380913A0290913B026AE070E05B
:100600000E94100B758364830E94370B8DB79EB7D1
:1006100006960FB6F8949EBF0FBE8DBF06C08AE146
:1006200092E06EE372E00E94480B19B110951078C9
:10063000C1F0EE20B1F42091380230913902C901A5
:1006400088199909069768F04901FF2019F05D9A09
:100650000ADE3DC0A4E0B0E0B0933D02A0933C02AE
:1006600002C0FF20A1F180913802909139028A19CD
:100670009B0920913A0230913B0282179307C0F107
:1006800080913C0290913D028F5F9340F0F4EDDD4C
:1006900028EE8039920711F46FEF03C06AE070E032
:1006A000D3D780913C0290913D020E944B0D8091E6
:1006B0003C0290913D02019690933D0280933C0252
:1006C000A0903802B090390213C0CDDD5D98FF24B0
:1006D00009C08091380283FF02C05D9801C05D9A15
:1006E000FF24F39480E292E04ED6C2D5E12E8FCE65
:1006F00080913C0290913D028F5F934050F3F0CF88
:10070000DC0120E040E050E098E115C0FD01E40F7D
:10071000F51FE08138E08E2F8227F82FF17080FDE1
:1007200029272695F13009F42068315011F0E6951B
:10073000F2CF4F5F5F4F4617570741F7822F08955B
:10074000382FDB0111969C91119780E02C91E22FBC
:10075000F0E0E82BF92B303181F4CF018E7F73E08C
:10076000880F991F7A95E1F716962C911697ECE071
:10077000F0E0E21BF109E80FF91FF7FD02C040E0CD
:1007800004C0F095E195FF4F41E0383211F032326C
:1007900099F414968C91282F30E020763070203216
:1007A000310539F02034310531F0232B29F4E87F6D
:1007B00003C0EC7F01C0EE7FCF018F70907060E8C6
:1007C00072E01CD7442311F480509E4F9C01232FCC
:1007D000332726952695CF0154E0969587955A950F
:1007E000E1F76AE070E00AD7280F391F442319F0B7
:1007F000309521953F4FC9018A5D9D4F89509740A3
:1008000010F020ED37E0C90108951F93CF93DF93D7
:10081000182FEB0191D08AD0882311F482E00AC00E
:10082000113021F084E4BE0155D103C084E4BE013F
:100830004FD180E0DF91CF911F910895EF92FF9209
:100840000F931F93CF93DF939C01062FF72EE42E77
:100850008EEBB9013DD1202F3F2DC901EC0110E0F5
:1008600003C0CBD089931F5F1E15D8F3802F9F2D17
:1008700069E070E045DF811183E0DF91CF911F9146
:100880000F91FF90EF900895CF92DF92EF92FF9239
:100890000F931F93DF93CF93CDB7DEB729970FB692
:1008A000F894DEBF0FBECDBF082F6B0180E090E053
:1008B0007E010894E11CF11CB70149E0BFDF182F4D
:1008C000882331F4802FB7013BDFF60191838083C9
:1008D000812F29960FB6F894DEBF0FBECDBFCF9102
:1008E000DF911F910F91FF90EF90DF90CF900895CF
:1008F0000F931F93CF93DF938C01EB01F80180815D
:10090000BE017DD0F801808381508D3F10F081E0E1
:1009100008C08881883221F0803111F0823271F76D
:1009200080E0DF91CF911F910F91089589B180747C
:1009300008955E9A569A08955E98569A80E897E0D0
:100940000197F1F78FB7F8945698E0E0F1E031970E
:10095000F1F729B18FBF80E896E00197F1F74E9942
:1009600002C081E00895822F807408950F931F9331
:10097000182F0FB7F894569A8AE08A95F1F711115B
:10098000569885E48A95F1F74E9B10E085EE8A959E
:10099000F1F75698662309F0CCDF0FBF85E38A95FF
:1009A000F1F7812F1F910F910895817060E0DECFE4
:1009B0000F931F93182F08E0812F8170F6DF169593
:1009C000811110680150C1F7812F1F910F91089577
:1009D0000F931F93182F08E0812F8170013011F0C1
:1009E00060E001C061E0C2DF16958111106801501E
:1009F00099F7812F1F910F9108958FEFD9CFDF9233
:100A0000EF92FF920F931F93CF93DF93E82EEB01AA
:100A100093DF882381F580EFCBDF80E4FF24182F5C
:100A200098EFD92ED80E81E0C0DF082F81E0BDDF1E
:100A3000882329F0002371F08EEFF82E1EC00023CA
:100A400049F41E1528F0888180FF04C0E11611F0DA
:100A5000F12E01E0802FA9DF88818695888300230D
:100A600011F08068888311501D15E9F6112329F0D3
:100A70002196812FD4CFFF24FA948F2DDF91CF912F
:100A80001F910F91FF90EF90DF900895FF920F93C9
:100A90001F93CF93DF93082FEB01F42E4DDF2097A8
:100AA00041F085E585DF18E0899182DF1150E1F79B
:100AB00002C08CEC7DDFFF2019F0802F89DF02C09F
:100AC000802F76DFDF91CF911F910F91FF900895D6
:100AD00040E0DCCF41E0DACFDA01923049F09330E8
:100AE00061F09130F9F4E4E7F0E022E130E01EC07B
:100AF000E6E8F0E02EE330E019C0813049F08130C3
:100B000018F0823079F408C0E4ECF0E0849107C07A
:100B1000E8ECF0E0849103C0E2EEF0E08491282F4D
:100B200030E004C0E0E0F0E020E030E0ED93FC9342
:100B3000C9010895382F282F2CC02093E9002317CE
:100B400021F4762F942F50E006C07091EC00909124
:100B5000ED005091F00091FF1BC08091EB008E7F63
:100B60008093EB008091ED008D7F8093ED0080916C
:100B7000EB0081608093EB007093EC009093ED00AC
:100B80005093F0008091EE0087FD02C080E0089550
:100B90002F5F253090F23093E90081E00895809135
:100BA000710288239CF404C0809170028823B9F0FC
:100BB0008091E80082FFF8CF8091E8008B778093E6
:100BC000E800089580917002882349F08091E80040
:100BD00080FFF8CF8091E8008E778093E800089539
:100BE0004091E4005091E50024E68091EC0080FF04
:100BF00024C08091E80080FD1EC08091700288238F
:100C000011F482E00895853011F483E00895809115
:100C1000EB0085FF02C081E008958091E40090918F
:100C2000E5008417950709F3222311F484E0089561
:100C30002150AC01DACF80E008958091E80082FF76
:100C4000DCCFF9CF41D043D08091D8008F7780930B
:100C5000D8008091D80080688093D8008091D80017
:100C60008F7D8093D80084E089BD86E089BD09B47A
:100C700000FEFDCF1092700210926C0210926E0274
:100C800010926D0280E060E042E054DF8091E1006C
:100C90008E7F8093E1008091E20081608093E2008A
:100CA0008091E20088608093E2008091E0008E7F76
:100CB0008093E0000895E3E6F0E080818E7F8083FA
:100CC00081E080936F02BECF1092E20008951092EF
:100CD000E10008951F920F920FB60F9211242F93E7
:100CE0003F934F935F936F937F938F939F93AF93B4
:100CF000BF93EF93FF938091E10082FF0AC0809140
:100D0000E20082FF06C08091E1008B7F8093E100CA
:100D1000AED28091E10080FF17C08091E20080FF99
:100D200013C08091E2008E7F8093E2008091E20008
:100D300080618093E2008091D80080628093D80027
:100D400019BC109270022CDA8091E10084FF2DC052
:100D50008091E20084FF29C084E089BD86E089BDDE
:100D600009B400FEFDCF8091D8008F7D8093D8001C
:100D70008091E1008F7E8093E1008091E2008F7E80
:100D80008093E2008091E20081608093E200809194
:100D90006C02882331F48091E30087FD02C081E07A
:100DA00001C084E080937002F6D98091E10083FF56
:100DB00022C08091E20083FF1EC08091E100877F06
:100DC0008093E10082E08093700210926C02809127
:100DD000E1008E7F8093E1008091E2008E7F80931E
:100DE000E2008091E20080618093E20080E060E0B8
:100DF00042E0A0DE3CD2FF91EF91BF91AF919F9175
:100E00008F917F916F915F914F913F912F910F90B3
:100E10000FBE0F901F9018959C0140917702509142
:100E200078024617570718F4F90190E03DC06115A4
:100E3000710511F0AB01F8CF8091E8008E778093B7
:100E4000E80040E050E0F0CF809170028823F1F19B
:100E50008530F1F18091E80083FF02C081E00895C0
:100E60008091E80082FD2CC08091E80080FF1CC0CA
:100E70008091F200282F30E007C081918093F1002B
:100E8000415050402F5F3F4F4115510519F0283018
:100E9000310598F390E02830310509F491E0809114
:100EA000E8008E778093E8004115510569F6992393
:100EB00059F606C080917002882341F0853041F0D8
:100EC0008091E80082FFF6CF80E0089582E00895E7
:100ED00083E008959C014091770250917802461773
:100EE000570718F4F90190E040C06115710511F041
:100EF000AB01F8CF8091E8008E778093E80040E066
:100F000050E0F0CF80917002882309F440C0853012
:100F100009F43FC08091E80083FF02C081E008959A
:100F20008091E80082FD2DC08091E80080FF1DC007
:100F30008091F200282F30E008C084918093F10066
:100F40003196415050402F5F3F4F4115510519F0E8
:100F50002830310590F390E02830310509F491E014
:100F60008091E8008E778093E8004115510551F695
:100F7000992341F606C080917002882341F08530A4
:100F800041F08091E80082FFF6CF80E0089582E092
:100F9000089583E008950F931F93DF93CF93CDB708
:100FA000DEB7AC970FB6F894DEBF0FBECDBFE1E75A
:100FB000F2E08091F100819322E0E937F207C9F76E
:100FC000F4D88091E80083FF39C18091710230919B
:100FD0007202353009F487C0363040F43130C9F13F
:100FE000313070F0333009F029C133C0383009F4A2
:100FF000F6C0393009F405C1363009F01FC197C079
:10100000803821F0823809F019C108C090916D0232
:1010100080916E02882399F0926011C080917502D0
:101020008F708093E9008091EB0090E025E0969529
:1010300087952A95E1F7982F91701092E900809199
:10104000E800877F8093E8009093F1001092F10010
:10105000D1C0882319F0823009F0F0C090E08F7180
:101060009070009721F0029709F0E8C00CC08091C1
:101070007302813009F0E2C010926E02333069F5DC
:1010800080936E022AC080917302882331F52091EB
:1010900075022F7009F4D2C02093E9008091EB0013
:1010A00080FF1BC0333021F48091EB00806213C0BD
:1010B0008091EB0080618093EB0081E090E002C0C2
:1010C000880F991F2A95E2F78093EA001092EA00B0
:1010D0008091EB0088608093EB001092E900809192
:1010E000E800877F8AC0882309F0A8C010917302A6
:1010F0001F770FB7F8948091E800877F8093E8000E
:101100004EDD8091E80080FFFCCF8091E300807885
:10111000812B8093E30080688093E300112311F416
:1011200082E001C083E0809370020FBF87C08058C7
:10113000823008F083C0809173029091740223E0A2
:101140008C3D920709F033C083E08C838AE28B8365
:101150007FB7F894DE0115966EE040E050E011E2B2
:10116000E62FF0E010935700849140FF03C0829572
:101170008F706F5F8F70282F30E08A3018F0C901B0
:10118000C79602C0C901C0968D939D934F5F5F4F74
:101190004431510529F77FBF8091E800877F809314
:1011A000E800CE0103966AE270E036DE12C060917C
:1011B0007502AE014F5F5F4F8FDCBC01009709F4F1
:1011C0003DC08091E800877F8093E80089819A8103
:1011D00081DE8091E8008B778093E8002FC0803813
:1011E00069F58091E800877F8093E80080916C0228
:1011F0008093F1008091E8008E778093E800CFDC47
:101200001DC08823D9F4909173029230B8F4809174
:10121000E800877F8093E80090936C02C0DC8091A7
:101220006C02882331F48091E30087FD02C081E0E5
:1012300001C084E0809370020E94D9008091E80090
:1012400083FF0AC08091EB0080628093EB00809165
:10125000E800877F8093E800AC960FB6F894DEBF75
:101260000FBECDBFCF91DF911F910F9108950895CB
:101270001F9380917002882361F01091E900109211
:10128000E9008091E80083FF01C085DE1F701093A4
:10129000E9001F910895FC0180917002843021F5CE
:1012A00081899289A389B4890097A105B105E1F0EC
:1012B00085818093E9008091E80082FF15C08091CC
:1012C000F200882319F42FEF3FEF04C08091F10062
:1012D000282F30E08091F200882341F48091E800CB
:1012E0008B778093E80002C02FEF3FEFC90108958C
:1012F000FB012EE0DB011D922A95E9F723E0238311
:1013000028EF39E0318720872BE839E033872287BF
:10131000958784870895FC0184859585BCDF9C01B1
:1013200097FF02C02EEF3FEFC90108950895FC0119
:1013300080917002843011F581899289A389B489E2
:101340000097A105B105D1F081818093E9008091DA
:10135000F2008823A9F09091E8008091E8008E7750
:101360008093E80095FD0CC03BDC982F882349F45E
:101370008091E8008E778093E80003C092E001C07E
:1013800090E0892F0895FC0180917002843051F41F
:1013900081899289A389B4890097A105B10511F0CB
:1013A000CF01C5CF08951F93FC01162F80917002C5
:1013B0008430D9F481899289A389B4890097A105E1
:1013C000B10599F081818093E9008091E80085FD65
:1013D00008C08091E8008E778093E80001DC8823C4
:1013E00029F41093F10080E001C082E01F9108957C
:1013F000282FFB0184859585622FD5DF882319F47A
:1014000020E030E002C02FEF3FEFC90108951F93A5
:10141000CF93DF93EC010D96FC018BE0DF011D9271
:101420008A95E9F711E08981181729F46A817B818F
:101430008C8152E010C08D81181731F46E817F814C
:10144000888552E030E008C08985181739F56A852B
:101450007B858C8553E030E8882311F440E001C09F
:1014600044E020E088E090E003C02F5F880F991FE0
:1014700086179707D0F3852F90E056E0880F991FC5
:101480005A95E1F760E0311161E0682B42602295E6
:10149000207F422B812F4EDB882329F01F5F1530E0
:1014A00009F0C1CF81E0DF91CF911F910895CF93D3
:1014B000DF93EC018091E80083FF9DC0888190E07C
:1014C00020917502309176022817390709F093C0F0
:1014D00080917202813269F0823220F4803209F008
:1014E0008AC03CC0823209F465C0833209F083C0EF
:1014F00074C080917102813A09F07DC08091E8004A
:10150000877F8093E8008091E80080FFFCCF898985
:101510009A89AB89BC898093F100292F3A2F4B2FF0
:1015200055272093F1009D01442755272093F10072
:101530008B2F9927AA27BB278093F1008D89809351
:10154000F1008E898093F1008F898093F100809162
:10155000E8008E778093E80022DB4DC08091710215
:10156000813209F048C08091E800877F8093E800CD
:101570008091E80082FFFCCF8091F1009091F10012
:101580002091F1003091F100898B9A8B2B8B3C8B51
:101590008091F1008D8B8091F1008E8B8091F10014
:1015A0008F8B8091E8008B778093E800F8DACE018A
:1015B000BDDE21C0809171028132E9F48091E800A2
:1015C000877F8093E800EBDA809173029091740238
:1015D0009E878D87CE01AADE0EC080917102813276
:1015E00051F48091E800877F8093E800D8DACE013B
:1015F000609173029BDEDF91CF91089555270024FF
:1016000080FF02C0060E571F660F771F6115710518
:1016100021F096958795009799F7952F802D08953D
:10162000AA1BBB1B51E107C0AA1FBB1FA617B70708
:1016300010F0A61BB70B881F991F5A95A9F7809524
:101640009095BC01CD01089597FB092E07260AD07D
:1016500077FD04D0E5DF06D000201AF4709561957F
:101660007F4F0895F6F7909581959F4F0895A0E0DC
:10167000B0E0ECE3FBE0CFC29E01275F3F4F8D81DE
:101680009E816F817885A9012BD02096E2E0DFC290
:10169000EF92FF920F931F93CF93DF937C018B0107
:1016A000DB0113968C9181FD03C0CFEFDFEF13C0F8
:1016B000C0E0D0E00BC0D8011896ED91FC911997CD
:1016C000B8010995892B11F0CFEFDFEFF701819178
:1016D0007F01882381F7CE01CDB7DEB7E6E0B3C244
:1016E000ABE0B0E0E5E7FBE086C24C012B015A011C
:1016F000FC0117821682838181FD03C06FEF7FEFAB
:10170000BEC11E010894211C311C9FE3692EF40107
:101710003381F20133FD859133FF81912F018823BD
:1017200009F4AAC1853239F433FD859133FF8191E3
:101730002F01853221F490E0B401D1D1E8CF982F68
:10174000FF24EE247724FFE1FF15D0F09B3269F0EF
:101750009C3228F4903259F0933291F40EC09D32AD
:1017600049F0903369F441E02AC052E0F52A84E060
:10177000F82A2EC098E0F92A2BC0E0E1FE2A28C002
:10178000F7FC2FC0292F20532A30A0F4F6FE08C002
:10179000872D90E06AE070E031DF782E720E18C07D
:1017A0008E2D90E06AE070E029DFE82EE20EF0E294
:1017B000FF2A0EC09E3229F4F6FC5EC140E4F42AF2
:1017C00007C09C3619F450E8F52A02C0983649F44F
:1017D000F20133FD959133FF91912F01992309F087
:1017E000B2CF892F8554833018F08052833030F483
:1017F00044E050E0A40EB51E69820FC0933631F06C
:10180000933779F0933509F052C01FC0F5018081FC
:10181000898342E050E0A40EB51E610101E010E0B2
:1018200011C0F501C080D180F6FC03C06FEF7FEFDF
:1018300002C0672D70E042E050E0A40EB51EC60164
:1018400043D18C015FE7F52213C0F501C080D18040
:10185000F6FC03C06FEF7FEF02C0672D70E042E03F
:1018600050E0A40EB51EC60124D18C0150E8F52A23
:10187000F3FE06C018C080E290E0B40130D1EA94D3
:101880008E2D90E008171907B0F30DC0F601F7FC94
:101890008591F7FE81916F0190E0B40120D1E110B4
:1018A000EA94015010400115110581F7E2C0943609
:1018B00011F0993661F5F7FE08C0F50120813181FC
:1018C0004281538184E090E00AC0F50180819181DA
:1018D0009C01442737FD4095542F82E090E0A80EEC
:1018E000B91E9FE6F92257FF09C0509540953095E3
:1018F00021953F4F4F4F5F4FE0E8FE2ACA01B901E3
:10190000A1012AE030E017D1D82ED2183FC0953778
:1019100029F41F2D1F7E2AE030E01DC01F2D197FE6
:101920009F3661F0903720F4983509F0A5C00FC0BC
:10193000903739F0983709F09FC004C028E030E0B4
:101940000AC0106114FD146020E130E004C014FDF1
:10195000166020E132E017FF08C0F5016081718157
:101960008281938144E050E008C0F501808191813B
:10197000BC0180E090E042E050E0A40EB51EA10161
:10198000DAD0D82ED2188FE7F82EF122F6FE0BC04F
:101990005EEFF522D71438F4F4FE07C0F2FC05C060
:1019A0008FEEF82202C01D2D01C0172DF4FE0DC0D0
:1019B000FE01ED0DF11D8081803319F499EEF922BD
:1019C00008C01F5FF2FE05C003C08F2D867809F0A6
:1019D0001F5F0F2DF3FC13C0F0FE0EC01E1510F09C
:1019E0007D2C0AC07D2C7E0C711A1E2D05C080E254
:1019F00090E0B40174D01F5F1E15C8F304C01E151B
:101A000010F4E11A01C0EE2404FF0EC080E390E060
:101A1000B40165D002FF1BC001FD03C088E790E060
:101A20000EC088E590E00BC0802F867881F001FF22
:101A300002C08BE201C080E2F7FC8DE290E0B401CD
:101A40004ED005C080E390E0B40149D07A94D71419
:101A5000C8F3DA94F101ED0DF11D808190E0B4013D
:101A60003ED0DD20B1F705C080E290E0B40137D070
:101A7000EA94EE20C9F74BCEF40166817781CB0161
:101A80002B96E2E1D4C0F999FECF92BD81BDF89AC0
:101A9000992780B50895262FF999FECF1FBA92BDD8
:101AA00081BD20BD0FB6F894FA9AF99A0FBE01963F
:101AB0000895FC010590615070400110D8F78095A1
:101AC00090958E0F9F1F0895FC016150704001900A
:101AD0000110D8F7809590958E0F9F1F08950F9352
:101AE0001F93CF93DF938C01EB018B8181FF1BC090
:101AF00082FF0DC02E813F818C819D81281739077F
:101B000064F4E881F9810193F983E88306C0E885EC
:101B1000F985802F0995892B31F48E819F8101965B
:101B20009F838E8302C00FEF1FEFC801DF91CF911B
:101B30001F910F910895FA01AA27283061F12031F1
:101B400091F1E8946F936E7F6E5F7F4F8F4F9F4F41
:101B5000AF4FB1E040D0B4E03ED0670F781F891F8F
:101B60009A1FA11D680F791F8A1F911DA11D6A0F61
:101B7000711D811D911DA11D22D009F468943F9112
:101B8000062E000C3019000C000C3019305D31931A
:101B9000CEF6CF010895462F4770405D4193B3E0E4
:101BA0000FD0C9F7F6CF462F4F70405D4A3318F07B
:101BB000495D31FD4052419302D0A9F7EACFB4E02C
:101BC000A6959795879577956795BA95C9F70097E4
:101BD0006105710508959B01AC010A2E0694579585
:101BE000479537952795BA95C9F7620F731F841FDC
:101BF000951FA01D08952F923F924F925F926F9272
:101C00007F928F929F92AF92BF92CF92DF92EF928C
:101C1000FF920F931F93CF93DF93CDB7DEB7CA1B0D
:101C2000DB0B0FB6F894DEBF0FBECDBF09942A8838
:101C3000398848885F846E847D848C849B84AA84E0
:101C4000B984C884DF80EE80FD800C811B81AA816D
:101C5000B981CE0FD11D0FB6F894DEBF0FBECDBF38
:081C6000ED010895F894FFCF97
:101C6800742020202073686F772074656D7065720A
:101C780061747572650D0A00632020202073686FF7
:101C8800772069737220636F756E7465720D0A0030
:101C9800682020202073686F7720656570726F6DEB
:101CA800206865616465720D0A0064202020207335
:101CB800686F7720656570726F6D20646174610D5F
:101CC8000A0031202020206461746120696E7465E7
:101CD8007276616C3A2031207365630D0A003520F5
:101CE8002020206461746120696E74657276616C6D
:101CF8003A20313620736563730D0A0036202020A0
:101D0800206461746120696E74657276616C3A2032
:101D1800333220736563730D0A0052656164206570
:101D280072726F720D0A0054656D703A2025642036
:101D38006465636963656C736975730D0A00436F45
:101D4800756E7465723A2025640D0A0053656373D5
:101D58003A2025643B20436F756E743A2025640D44
:101D68000A00256420000D0A446F6E650D0A007391
:101D78006563733A2025640D0A000D0A3F0D0A00B9
:101D8800000310000004100000020800000000001A
:081D9800000000000000000043
:00000001FF
